:1000000000308A005F2A0000FF00030E8301A10078
:100010007F08A0000A08A8008A01A00E0408A20018
:100020007708A3007808A4007908A5007A08A6003C
:100030007B08A700831383128C308400801D222844
:100040008C1939288B1E26280B193B28220884007E
:100050002308F7002408F8002508F9002608FA000C
:100060002708FB0028088A00210E8300FF0E7F0E60
:1000700009008A11A5288A11D3280A108A100A11AA
:100080008207023406340E341E343E347E34FE348D
:10009000FF340A108A100A1182070C344D346F3471
:1000A000643465343A342534643400340A108A10D8
:1000B0000A1182070A34503457344D343A34253407
:1000C0003034333475342034523455344E343A3469
:1000D000253430343334753400340A108A100A1150
:1000E00082070A34523455344E343A34253433348A
:1000F00075346D347334203400340A108A100A11B8
:1001000082070A3441344C3447343A34253430348D
:10011000333475342034253430343334753420345A
:10012000253430343334753400340A108A100A11FF
:1001300082072034523455344E343A342534333423
:1001400075346D347334203400342A0893008C11D4
:100150008A112628C508031DB928831606118312A3
:100160000611831694018312940183168C11D128F1
:1001700083124508073C0318BF280830C500C50393
:1001800045083D20F800AA008316061183120611C7
:10019000831694012230831294002A089300831658
:1001A0008C15831200342B082C040319DB282B0830
:1001B0000319AC03AB03AD08031DAD03AF0803196E
:1001C000EE282F08073C031CEE28AD08031DEE287F
:1001D0002E08AD00AF0A2F08C500AA200B118A1106
:1001E00026281A3083169900803083129800243014
:1001F0008316980083128A118C2A1130BF02031CC7
:100200000F293F308400FC3080050310800C800CE7
:10021000000803190F290D296400800B0C298A118D
:10022000AA2A8316981816298312112983124208C4
:10023000990000344308F8014202031822294208B9
:10024000F7002E29F7010830C400C20DF70D43084E
:1002500077020318F700F80DC40B25290034BF1FDF
:100260003529C017BF09BF0A3C29401D3C29203051
:10027000401E3030C20011214013C0123F08C2009E
:100280006430C3001A217708BF007808031D66296F
:10029000C01A6629C0197429401B542940185429D2
:1002A00040195429C01B7429401C6029C01B7429A3
:1002B000401B60294018742940196029C01B74290B
:1002C0002030401E3030C20011217429C016C01FDA
:1002D000702978088000F8002D30C2001121C01369
:1002E00030307807C2001121401B7F293F08C2002F
:1002F0000A30C3001A217708BF0040174529C01FE4
:1003000084292D30C200112130303F07C200112155
:100310008A11D12A83160108C0390138810083125D
:100320008B16C0308B048A11DF2A3E08043C031D63
:100330009D298316861083128614303083169F0001
:1003400083123E0DF700F70DF70DF830F70577082B
:10035000413E9F0064001030F700F70BAD2900000C
:1003600000001F1564001030F700F70BB5290000DE
:10037000000083168610831286101E08F8000034D1
:100380004113C1124008C2006430C3001A2177082B
:10039000C0007808031DEA29C11AEA29C119F82901
:1003A000411BD8294118D8294119D829C11BF8293E
:1003B000411CE429C11BF829411BE4294118F829F3
:1003C0004119E429C11BF8292030411E3030C200F8
:1003D0001121F829C116C11FF42978088000F800FE
:1003E0002D30C2001121C11330307807C200112115
:1003F000411B032A4008C2000A30C3001A217708B3
:10040000C0004117C929C11F082A2D30C20011217F
:1004100030304007C200112100343E308400000813
:100420000319232A0130F800BF30F7006400F70BEE
:10043000162AF80B142A5830F700F70B1D2A000073
:100440006400800B122A0034A9018B1BA9178B139F
:100450003E08C500AA20A91B8B17C0308B040034AE
:100460008B123F08AC003E08AB008B1600348B1299
:10047000AB08031D3E2AAC080319402A0030412A6C
:100480000130F8007818462A3E10472A3E148B1691
:1004900000303E180130F80000348B120130AF00FC
:1004A0003E08AE002E08AD008B16A9018B1BA917C4
:1004B0008B130130C500AA20A91B8B1700348401BF
:1004C0001F30830583161F129F121B0880399B0063
:1004D00007309C001C0883120D13623083168F00B6
:1004E0008611831286118316061183120611831654
:1004F0008610831286108316061283120612831644
:10050000811381110E308312031785001F3083166B
:1005100003139B008312F1280130B10031081D3C08
:10052000031CAE2A3218962A0513972A051783163C
:10053000051301308312B2063218A02A8513A12AAE
:10054000851783168513640009308312BE006C3052
:10055000BF00FD28BE0BA72AB10A8E2AB001831660
:1005600086178312861F3014831606178312061F00
:10057000B014831686138312861383160613831210
:100580000613BE013E084920BE0AF700C200112131
:1005900006303E02031DC22A3008BF001830C000DA
:1005A0002F291F30831692000430831292000C30E2
:1005B0009700950183168611831286118A29300BC4
:1005C0001A2B6400BE0195217808B300B30CB30C5C
:1005D0003F30B3050130BE0095217808B400B40E59
:1005E0000F30B405BE013E085620BE0AF700C20017
:1005F000112105303E02031DF32A3308C000C1015A
:10060000C0210930BF003F085620BF0AF700C200D2
:1006100011210E303F02031D032B3408C000C1011D
:10062000C0211430BE000D22330895003408BE00EE
:100630002422E12A3008023C031D6B2BB601013055
:10064000BE0095217808B500BE013E086D20BE0AA7
:10065000F700C200112105303E02031D252B35088D
:10066000C0001030C100C0216D30C20011217330B4
:10067000C20011212030C20011210A30BE000D221B
:10068000B608031D492BB60A0730BF00D030BE00A4
:100690003022360B5B2B3722F80803195B2BB60A86
:1006A0005230C20011213508BE004D220730BF0074
:1006B000D030BE0030223608023C031D692B3722A1
:1006C000F8080319692BB60A5330C2001121BE0184
:1006D000242264001F2B3008033C031DC22BB701EA
:1006E0006400BE0195217808B800BE019521031071
:1006F000780C323EB8000430BE0095217808B9006D
:10070000380839020318882B37081D3C0318B70A2C
:1007100038083902031C8F2BB708031DB7030A30B2
:10072000B907380839020318992B37081D3C0318FC
:10073000B70A3708183C03189F2B1830B700370842
:100740009500BE013E087D20BE0AF700C2001121BF
:1007500005303E02031DA22B3808C000C101C02194
:100760002030C20011213908C000C101C021203051
:10077000C20011213708C000C101C0210A30BE00EB
:100780000D22702BB008031D492C0130BE009521AD
:100790007808BD00BE013E089520BE0AF700C200E1
:1007A000112105303E02031DCB2B3D08C000103047
:1007B000C100C0216D30C20011217330C20011216F
:1007C0002030C20011210A30BE000D22BA0136309D
:1007D000BF00B030BE003022B2146400BE019521CB
:1007E0007808BB00BE0195210310780C323EBB0097
:1007F0000430BE0095217808BC003B083C02031879
:10080000052C3A081D3C0318BA0A3B083C02031C9D
:100810000C2CBA08031DBA030A30BC073B083C0283
:100820000318162C3A081D3C0318BA0A3A08183C5B
:1008300003181C2C1830BA003A089500BE013E0877
:100840007D20BE0AF700C200112105303E02031DC3
:100850001F2C3B08C000C101C0212030C200112163
:100860003C08C000C101C0212030C20011213A085B
:10087000C000C101C0210A30BE000D223722F80895
:100880000319482CB21C482CB2103D08BE004D2262
:04089000ED2B6300E9
:04400E003C2FFF3F05
:00000001FF
